:020000041000EA
:400000000001000831010010000000000000000000000000000000000000000000000000000000000000000000000000000000000000000000000000000000000000000075
:400040000000000000000000000000000000000000000000000000000000000000000000000000000000000000000000000000000000000000000000000000000000000080
:400080000000000000000000000000000000000000000000000000000000000000000000000000000000000000000000000000000000000000000000000000000000000040
:4000C0000000000000000000000000000000000000000000000000000000000000000000000000000000000000000000000000000000000000000000000000000000000000
:40010000526F736574746120636F646500000000764FAF5C61AC315F1497F9DFA542713965B785E5CC2F707D6468D7D1124CDFCF13B500240C4800F01DF821000094012395
:4001400006220A4800F062F80123009406221900064800F05BF801340222044B0448DC60DA6000F099F8F7E7280300108000324020BCBE00014B18607047C0463C100008CC
:4001800070B50D00044C01001822200000F094F8A56101BEFEE7C0460010000870B506000C001500072903D914491548FFF7E8FF1F232A009A4303D012491148FFF7E0FF8A
:4001C000114B1B689A695B69B01AC0090001C0181F231D40032C07D8E400A340A54002689A431543056070BD043CE400A340A54042689A4315434560F5E7C04642020000CD
:4002000033040010430200003C100008F7B51D0008AB1B7807000E0014000193072903D9D1211B48FFF7ACFF0F2322009A4303D0D2211748FFF7A4FF012D03D9D3211448C7
:40024000FFF79EFF1F23019A9A4303D0D4211048FFF796FF012211001540B140B5400F203B6804408B431D433D600500B1008D408C40084B31001B68380063331A78BA18AE
:400280001368AB431C431460019AFFF787FFF7BD100400103C1000080230800803D001300238FCD1C046C0467047EFF3108072B6704780F310887047000052E3011041E2BB
:4002C00000C0A0E11EFF2F0110402DE90C30A0E101E0F1E500005EE3014042E201E0C3E40400001A02C08CE00C0053E10500000A01E0C3E4FBFFFFEA000054E303C0A0E1E7
:400300000420A0E1F0FFFF1A1040BDE81EFF2FE10DC0A0E1F8DF2DE904B04CE20DC0A0E1F8DF2DE904B04CE200002140000025400000014000003440000024400000314064
:400340000000324000001F4101010101010101010110101080550501053B04101C0101000FC000000000100001010101011D3A577896000820000010000F002000023F06D7
:40038000080E00080009000A000B24282C303400100000009000000088000000080000008000000004F0000000F000002005A000D00100018001A0011000000004000000C4
:4003C000400000004400000048000000800000000001000010020000880200000004000010040000200400004004000048040000800400008404000090040000C0070000E1
:40040000C4070000C8070000CC070000004000002E2F68616C2F70646C2F647269766572732F736F757263652F63795F6770696F2E63002E2F68616C2F70646C2F64726907
:40044000766572732F696E636C7564652F63795F6770696F2E68000000000000000000000000000000000000000000000000000000000000000000000000000000000000FA
:40048000000000000000000000000000000000000000000000000000000000000000000000000000000000000000000000000000000000000000000000000000000000003C
:4004C00000000000000000000000000000000000000000000000000000000000000000000000000000000000000000000000000000000000000000000000000000000000FC
:4005000000000000000000000000000000000000000000000000000000000000000000000000000000000000000000000000000000000000000000000000000000000000BB
:40054000000000000000000000000000000000000000000000000000000000000000000000000000000000000000000000000000000000000000000000000000000000007B
:40058000000000000000000000000000000000000000000000000000000000000000000000000000000000000000000000000000000000000000000000000000000000003B
:4005C00000000000000000000000000000000000000000000000000000000000000000000000000000000000000000000000000000000000000000000000000000000000FB
:0200000490303A
:02000000FF3BC4
:0200000490501A
:0C00000000000000000000000000FF3BBA
:00000001FF
